:100000000C9478050C9495050C9495050C94950525
:100010000C9495050C9495050C9495050C949505F8
:100020000C9495050C9495050C9468260C943A272D
:100030000C94B1200C9495050C9495050C949505A1
:100040000C9495050C9495050C9495050C949505C8
:100050000C9495050C9439210C9495050C949505F8
:100060000C9495050C9495050C9495050C949505A8
:100070000C9495050C9495050C9495050C94950598
:100080000C9495050C9495050C9495050C94950588
:100090000C9495050C9495050C9495050C94950578
:1000A0000C9495050C9495050C949505DB08DB08DC
:1000B000070907096F098D09A50AA50A9809310AD8
:1000C000420A420AA727CE27C628CE27C6281A28C2
:1000D0003D28C6289428A32829001E001F002000C0
:1000E00021002200230024002500260027002D00E7
:1000F0002E002A004A002B0014001A0008001500E8
:1001000017001C0018000C00120013002F00300014
:1001100031004D00390004001600070009000A00F4
:100120000B000D000E000F0033003400000028000B
:100130004B00E1001D001B00060019000500110026
:100140001000360037003800E500000052004E0075
:10015000E000E300E200000000002C0000000000CE
:100160000000E6000151E400500051004F0035004E
:100170003A003B003C003D003E003F004000410093
:1001800042004300440045004C0001000100010012
:100190000100010001000100010001000100010057
:1001A0000100460047004800010001000100010075
:1001B0000100010001000100010001000100010037
:1001C0000100000001000100010001000100010028
:1001D0000100010001000100010001000100010017
:1001E000000001000100005C0100010000000000AF
:1001F00001000000000000000100010001000100FA
:100200000100010044454255473A20646973616228
:100210006C65642E0A0044454255473A20656E617C
:10022000626C65642E0A000A0025303258006C6545
:10023000645F7461736B3A20004F6E6573686F740E
:100240003A206163746976653A2025640A000A00E1
:100250002530313662003A200025303258000A72CB
:100260002F63203031323334353637383941424309
:100270004445460A00290A002575002F002575000F
:100280005D2800256400200025640020002564000E
:1002900020002564007C0025303258006D6F757396
:1002A000656B6579205B62746E7C7820792076209E
:1002B000685D287265702F61636C293A205B00319C
:1002C0003A0964656C6179282A31306D73293A20C6
:1002D00025750A323A09696E74657276616C286D0B
:1002E00073293A2025750A333A096D61785F737076
:1002F0006565643A2025750A343A0974696D655F4D
:10030000746F5F6D61783A2025750A353A09776810
:1003100065656C5F6D61785F73706565643A202513
:10032000750A363A09776865656C5F74696D655F53
:10033000746F5F6D61783A2025750A00703A097014
:1003400072696E742076616C7565730A643A09731C
:1003500065742064656661756C74730A75703A091A
:100360002B310A646E3A092D310A6C743A092B312B
:10037000300A72743A092D31300A4553432F713ACD
:1003800009717569740A0A7370656564203D20649B
:10039000656C7461202A206D61785F737065656497
:1003A000202A2028726570656174202F2074696D81
:1003B000655F746F5F6D6178290A77686572652083
:1003C00064656C74613A20637572736F723D256465
:1003D0002C20776865656C3D25640A536565206847
:1003E0007474703A2F2F656E2E77696B697065642F
:1003F00069612E6F72672F77696B692F4D6F757307
:10040000655F6B6579730A004D3E20004D25753A96
:1004100025733E20003F0A003D2025750A003F0A53
:100420000064656661756C74730A0025750A003F87
:100430000A000A092D2056616C756573202D0A008B
:10044000710A000A092D204D6F7573656B6579205F
:100450002D0A003F00433E20004C25640A000A0993
:100460002D20537461747573202D0A686F73745F47
:100470006B6579626F6172645F6C65647328293A99
:1004800020253032580A6B6579626F6172645F7043
:10049000726F746F636F6C3A20253032580A6B6547
:1004A00079626F6172645F69646C653A20253032ED
:1004B000580A74696D65725F726561643332282908
:1004C0003A202530386C580A000A092D20566572EA
:1004D00073696F6E202D0A5649443A2030783737B9
:1004E000363728416C697347726176654E696C29AD
:1004F000205049443A2030783843373828546865CA
:1005000020536564616E29205645523A2030783078
:100510003030310A4255494C443A20202846656221
:100520002032372032303232290A4F5054494F4E50
:10053000533A204C554641204D4F5553454B455954
:100540002045585452414B455920434F4E534F4C30
:100550004520434F4D4D414E4420343039360A47F3
:1005600043433A20352E342E30204156522D4C49EB
:1005700042433A20322E302E30204156525F4152B3
:1005800043483A20617672350A000A092D20436FEC
:100590006E736F6C65202D0A4553432F713A0971B4
:1005A0007569740A6D3A096D6F7573656B65790AC3
:1005B000000A092D204D61676963202D0A443A091C
:1005C0004465627567204D65737361676520546F7C
:1005D00067676C650A583A094D61747269782044FE
:1005E00065627567204D6F646520546F67676C6541
:1005F000202D2053686F77206B6579707265737357
:10060000657320696E206D61747269782067726904
:10061000640A4B3A094B6579626F617264204465E4
:1006200062756720546F67676C65202D2053686F73
:1006300077206B65797072657373207265706F7265
:10064000740A4D3A094465627567204D6F7573658C
:1006500020546F67676C650A563A0956657273696C
:100660006F6E0A533A095374617475730A433A09F9
:10067000416374697661746520436F6E736F6C6556
:10068000204D6F64650A46312D4631303A09537763
:100690006974636820746F204C6179657220302D15
:1006A000392028463130203D204C30290A302D3960
:1006B0003A0953776974636820746F204C617965D7
:1006C0007220302D390A47524156453A095377690D
:1006D00074636820746F204C617965722030202823
:1006E000616C7465726E617465290A423A094A75D3
:1006F0006D7020746F20426F6F746C6F61646572EF
:100700000A4553433A094A756D7020746F20426F51
:100710006F746C6F616465722028616C7465726EB1
:10072000617465290A453A095072696E742045451D
:1007300050524F4D2053657474696E67730A42536B
:10074000504143453A09436C65617220454550521A
:100750004F4D0A006B65796D61705F636F6E6669FE
:10076000672E7261773A20253032580A2E737761EE
:10077000705F636F6E74726F6C5F636170736C6FC8
:10078000636B3A2025750A2E636170736C6F636B1F
:100790005F746F5F636F6E74726F6C3A2025750AB9
:1007A0002E737761705F6C63746C5F6C6775693A08
:1007B0002025750A2E737761705F7263746C5F72A7
:1007C0006775693A2025750A2E737761705F6C61D1
:1007D0006C745F6C6775693A2025750A2E737761B2
:1007E000705F72616C745F726775693A2025750A73
:1007F0002E6E6F5F6775693A2025750A2E737761D3
:10080000705F67726176655F6573633A2025750A6C
:100810002E737761705F6261636B736C6173685F85
:100820006261636B73706163653A2025750A2E6E91
:100830006B726F3A2025750A0064656275675F63A5
:100840006F6E6669672E7261773A20253032580ADA
:100850002E656E61626C653A2025750A2E6D617495
:100860007269783A2025750A2E6B6579626F61721C
:10087000643A2025750A2E6D6F7573653A202575CB
:100880000A006565636F6E6669673A0A646566614A
:10089000756C745F6C617965723A2025750A003F4A
:1008A000000A6D6F7573653A206F66660A000A6DFF
:1008B0006F7573653A206F6E0A000A6B6579626F17
:1008C0006172643A206F66660A000A6B6579626F2E
:1008D0006172643A206F6E0A000A6D617472697801
:1008E0003A206F66660A000A6D61747269783A2070
:1008F0006F6E0A000A64656275673A206F66660A61
:10090000000A64656275673A206F6E0A000A0A4A37
:10091000756D70696E6720746F20626F6F746C6F95
:10092000616465722E2E2E2000433E2000436C65CC
:100930006172696E6720454550524F4D0A000A00AA
:100940002530325820006B6579626F6172645F7286
:1009500065706F72743A20005B735D005B575D00D9
:100960005B535D005B525D005B445D005B435D007B
:100970001403540068006500200053006500640003
:1009800061006E0000001A0341006C0069007300F2
:10099000470072006100760065004E0069006C003F
:1009A00000000403090409025B00030100A0FA0926
:1009B000040000010301010009211101000122408E
:1009C000000705810308000109040100010300007C
:1009D00000092111010001227B000705820320008C
:1009E00001090402000203000000092111010001B5
:1009F00022220007058303200001070503032000CE
:100A00000112010002000000086777788C010001E4
:100A10000200010631FF0974A1010975150026FFC6
:100A2000009520750881020976150026FF009520A3
:100A300075089102C005010902A10185020901A101
:100A4000000509190129081500250195087501817E
:100A5000020501093009311581257F95027508814C
:100A60000609381581257F950175088106050C0A50
:100A700038021581257F950175088106C0C00501E2
:100A80000980A101850319012AB700150126B700C5
:100A9000950175108100C0050C0901A1018504199B
:100AA000012AA002150126A002950175108100C03F
:100AB00005010906A101050719E029E7150025012F
:100AC00095087501810295017508810105071900D6
:100AD00029FF150026FF00950675088100050819F5
:100AE000012905950575019102950175039101C0D4
:100AF00011241FBECFEFDAE0DEBFCDBF11E0A0E0D2
:100B0000B1E0E8E0F3E502C005900D92AC3FB1071B
:100B1000D9F722E0ACEFB1E001C01D92A23FB207CD
:100B2000E1F70E9408170C9482290C940000FF93AF
:100B3000EF93E091FC01F091FD01309709F00995E8
:100B4000EF91FF910895FC018591803011F0EFDF66
:100B5000FBCF0895FF27E0E230E247FF0CC041954C
:100B600097FF09C0EDE26095709580959095611DA5
:100B7000711D811D911D27FF02C0219530E350E2B8
:100B8000AA27660F771F881F991FAA1FA41710F0A6
:100B9000A41B63955A95A9F7AA3008F0A95FA05D38
:100BA000AF93F395611571058105910541F7ED321C
:100BB00011F4EF93F395F21718F43F93F395FBCFED
:100BC0008F91B5DFFA95E1F70895E991F991859153
:100BD000803021F0853219F0AADFF9CF089520E0A6
:100BE000E89455915532C1F3503311F468945591FE
:100BF0005A3348F4505390F3220F022E220F220F43
:100C0000200D250FF4CF0EF421958991999153363B
:100C100019F3533729F1533559F1BC018827992726
:100C2000E8945C3621F489919991689455915436F1
:100C300039F446EF7EF077FF0DC08FEF9FEF0AC0CB
:100C400055374AE039F0583540E121F0523642E05C
:100C500009F00895FF93EF937DDFEF91FF91B7CFF8
:100C6000FF93EF93FC0181918030B9F360DFFBCFFC
:100C7000FF93EF9368DFF1CFDF93CF93CDB7DEB76C
:100C80002596A3DFCF91DF91089581E0089581E05B
:100C900008950C94470608950C944B061F93CF9328
:100CA000DF9300D000D01F92CDB7DEB749835A83BF
:100CB0006B833091FF0189819A81311114C06623C1
:100CC00059F0222349F00E94E20C182F682F8981E5
:100CD0009A810E948B0C03C00E94B60C182F698168
:100CE0007A81812F04C00E94E20C69817A810F9081
:100CF0000F900F900F900F90DF91CF911F910C9458
:100D00002C14FC01262F40815181628173818481E2
:100D10000C944E0681E00895CF93DF93EC0160E0E0
:100D20000E948106BE01DF91CF910C944C060C9479
:100D3000B9150C94B51508950E94350B0E949B06B9
:100D40002FEF84E39CE0215080409040E1F700C009
:100D500000000C945F210F931F93CF93DF938C01BE
:100D600061E00E948106EC01B8010E9449068823D7
:100D700009F45BC0B801CE010E943E1F882309F42C
:100D800054C0B801CE010E94201A882309F44DC036
:100D9000B801CE010E949A1E882309F446C0F801CA
:100DA00082818823D9F1CF3D8CE5D80779F140F4D1
:100DB000C115FCE5DF0791F0C130DC4591F02EC094
:100DC000CC35EDE5DE0741F1CD35FDE5DF0709F175
:100DD000CB35DD4519F50E94791120C00E949C0693
:100DE00024C080919802C82FC095C170C0FB80F9C3
:100DF00080939802CC2329F086E192E00E94A3051B
:100E000014C084E092E00E94A30510C00E942D123D
:100E10000CC00E94701102C00E947C11C801DF91B9
:100E2000CF911F910F910C944506C0E08C2FDF915C
:100E3000CF911F910F9108950E9493200C945A070F
:100E40000E945D070C9499208295982F937344E03B
:100E5000949F900111248C7C86958695282B822F57
:100E60008575880F2A7A2695822B0895CF93DF9374
:100E7000D92F0E942407C82F8D2F0E9424072C2FC2
:100E800030E0322F2227A901482BCA01DF91CF91F0
:100E9000089508950C94490781E008950C944C0737
:100EA0000895CF93C82F0E944A078C2F0E944E07A7
:100EB000CF91089580E00C9451070E949A1F0C94E2
:100EC0005107CF930E949A1FC82F8091FE01C81727
:100ED00041F1C093FE018091980282FF1EC080FF05
:100EE00004C08EE292E00E94A3058091980280FFE8
:100EF0000CC01F92CF9389E292E09F938F930E9440
:100F00003C060F900F900F900F908091980280FFF9
:100F100004C087E292E00E94A3058C2FCF910C942D
:100F20005107CF910895CF93DF93CDB7DEB72B97BD
:100F30000FB6F894DEBF0FBECDBF4F8358876987C9
:100F40007A878B8761110E94A8109E012F5F3F4F07
:100F500086E0F90111928A95E9F785E0FE0137965E
:100F6000D90101900D928A95E1F789819A814C818E
:100F70005D81452B31F09F3F31F491E08F3F19F4B3
:100F800003C091E001C090E090FF09C049815A81FF
:100F90006B817C818D819E810E94C90F05C0C90132
:100FA0000E948A068111F2CF2B960FB6F894DEBF0D
:100FB0000FBECDBFDF91CF910895FC01808191815B
:100FC0000E94240D0895CF93882309F455C0C82F9B
:100FD0008CEF8C0F813AF8F48C2F0E94431E811104
:100FE0004BC06C2F80910201909103010E9435202B
:100FF000882349F06C2F80910201909103010E9497
:101000006D200E94CA106C2F809102019091030103
:101010000E946B200CC080E28C0F883058F4C7709F
:1010200081E001C0880FCA95EAF70E948B10CF912A
:101030000C94CA10EBE5EC0FE33040F4F0E0E95B10
:10104000FE4F808190E0CF910C94FD1FE8E5EC0FFE
:10105000E73150F4F0E0EE0FFF1FE75EFE4F8081B6
:101060009181CF910C941320CD3E30F08C2F0E94B3
:101070008D17CF910C945F18CF910895882389F133
:101080009CEF980F913A40F4682F80910201909163
:1010900003010E946D200DC090E2980F983058F423
:1010A000877091E001C0990F8A95EAF7892F0E9415
:1010B00091100C94CA109BE5980F933020F480E0B7
:1010C00090E00C94FD1F98E5980F973120F480E094
:1010D00090E00C9413208D3E20F00E94E8170C94B1
:1010E0005F1808951F93CF93DF93182FEB010E9491
:1010F000E307209741F08FE99FE00197F1F700C0E7
:1011000000002197F6CF812FDF91CF911F910C9492
:101110003E08893319F060E070E002C060E570E0DD
:101120000C947208882321F00E948B100C94CA1032
:101130000895882321F00E9491100C94CA100895FC
:10114000CF92DF92EF92FF920F931F93CF93DF9393
:101150007C01D62FC72FFC011281058102950F70EB
:101160000E9481108823B9F01123A9F08C2F807F71
:10117000803421F080E28D0F883068F08091CC02BD
:1011800082FD09C082E00E942A110E94811091E034
:10119000D82ED92601C0D12CCC2EC2948FE0C822E3
:1011A0008C2D90E08C30910508F0CFC1FC01EA5AFB
:1011B000FF4F0C9419298C2F807FCF70882311F05A
:1011C000C295C07F112399F0CC2309F4AAC180E213
:1011D0008D0F883010F0D11104C08C2F0E948B101D
:1011E00003C08C2F0E949B100E94CA109AC18D2FA1
:1011F0000E943E08CC2309F4A8C180E28D0F8830FC
:1012000038F1DD2329F18C2F0E94A11024C08C2FEE
:10121000807FCF70803211F0C295C07FDD2319F03E
:10122000D130A1F13DC08091CC0282FF17C01123C3
:1012300049F0CC2329F08C2F0E948B100E94CA10F9
:1012400080E070C180E00E943E08CC2309F47DC19B
:101250008C2F0E9491100E94CA1077C1112371F047
:10126000002341F0013031F40E94AB108C2B0E941E
:10127000B3106BC10E94AB108C2B1DC0002319F062
:10128000013009F462C10E94C01025C0112321F071
:10129000063008F05AC10EC0053008F056C11BC018
:1012A000112361F0002331F0F701858180FF39C1FE
:1012B0008F7085838C2F0E94920847C1002359F0BC
:1012C000D93309F03FC1FFEF07EE13E0F1500040C2
:1012D0001040E1F735C18C2F0E94990836C18C2F40
:1012E00086958695837019F0813061F02EC11123A7
:1012F00021F08D2F9C2F937002C080E090E00E941F
:10130000FD1F2BC1112321F08D2F9C2F937002C044
:1013100080E090E00E94132020C18D2F112319F04E
:101320000E948D1702C00E94E8170E945F1815C125
:101330008C2F837009F047C011110BC12D2F2295FE
:1013400026952770220F220F6D2F6F70862F90E049
:10135000A0E0B0E0022E04C0880F991FAA1FBB1F97
:101360000A94D2F7D4FF10C04FE050E060E070E084
:1013700004C0440F551F661F771F2A95D2F740956A
:1013800050956095709503C040E050E0BA01C69555
:10139000C695C3708A019B01082B192B2A2B3B2B66
:1013A000C901B801C23049F058F4C13019F00E94A7
:1013B000A10BCFC00E948F0BCCC00E94B30BC9C041
:1013C0000E948D0BC6C0112319F08C2F817001C0B3
:1013D0008695882309F4BDC02D2F22952695277068
:1013E000220F220F6D2F6F70862F90E0A0E0B0E0EB
:1013F000022E04C0880F991FAA1FBB1F0A94D2F7A0
:10140000D4FF10C04FE050E060E070E004C0440F33
:10141000551F661F771F2A95D2F740955095609506
:10142000709503C040E050E0BA01C695C695C37000
:101430008A019B01082B192B2A2B3B2BC901B801D0
:10144000C23049F058F4C13019F00E94660C81C0D6
:101450000E94540C7EC00E94780C7BC00E94C70B77
:1014600078C0CF70112339F08C2F0E94ED0B8D2F97
:101470000E9492086EC08D2F0E9499088C2F0E94A6
:101480000E0C67C0D23F21F128F4D03F41F0D13F8C
:10149000C1F043C0D33F19F1D43F79F03EC01123CE
:1014A00041F0053008F051C08C2F8F710E94330C31
:1014B0004CC0063008F049C0F7CF8091CC0282FFC3
:1014C00018C0112339F08C2F8F710E94ED0B3DC095
:1014D0001123C9F38C2F8F710E940E0C36C011237B
:1014E00029F08C2F8F710E94D80B2FC00E94D30B34
:1014F0002CC0112349F0CF718C2F0E94ED0B63E0BB
:101500008C2F0E940F1121C081E00E942A1102300D
:10151000E0F082E00E942A1118C0112331F000236C
:1015200091F28D2F0E94E30710C0002399F2D93366
:1015300049F41FEF27EE33E0115020403040E1F72F
:1015400000C000008D2F0E943E0888EF8C0D843073
:1015500020F40E949A1F0E945107DD20C9F00E94CA
:101560007D1080FD15C0F70112820E9477100E9445
:10157000ED0BC7010E94E90A0E947710DF91CF911D
:101580001F910F91FF90EF90DF90CF900C940E0C75
:10159000DF91CF911F910F91FF90EF90DF90CF904F
:1015A00008950F931F93CF93DF93EC0168817981A6
:1015B0008A810E942F0D8C010E948A0C0E947B0B55
:1015C000B801CE010E94A008DF91CF911F910F9129
:1015D0000895CF93DF93EC01988189812B813C8121
:1015E000232B31F08F3F31F481E09F3F19F403C08A
:1015F00081E001C080E080FD1DC0CE010E94AB06ED
:10160000811110C00E9481108823A1F08A81882353
:1016100089F08091CC0282FD0DC082E0DF91CF91F4
:101620000C942A11CE010E94D10ACE01DF91CF91F4
:101630000C948C06DF91CF91089580E090E00E9499
:10164000FD1F80E090E00E9413200E94A8100E94DD
:10165000CA100E94121A0C945F1880910201909196
:1016600003010E946F200C941D0B0E9498100C9493
:101670002D0B92959F70963079F010F4925001C026
:101680009A50923068F4803F69F018F4883E40F434
:1016900009C0843F29F406C0883E20F0813F11F044
:1016A00080E0089581E00895FC01808191810E948D
:1016B000240D0E94390B0895CF93DF9300D000D002
:1016C0001F92CDB7DEB70F900F900F900F900F9035
:1016D000DF91CF910895CF93DF9300D000D000D059
:1016E000CDB7DEB726960FB6F894DEBF0FBECDBFDE
:1016F000DF91CF910895089508950C947C0B0C947C
:101700007D0B0E947F0B60933602709337028093AB
:101710003802909339020C941D0B0C94810B0F939B
:101720001F930091360210913702209138023091B8
:101730003902602B712B822B932B1F910F910C94EC
:10174000810B0F931F930091360210913702209165
:1017500038023091390260237123822393231F9131
:101760000F910C94810B0F931F93009136021091EF
:101770003702209138023091390260277127822781
:1017800093271F910F910C94810B0C947C0B0E945A
:10179000C50B6093320270933302809334029093AE
:1017A00035020C941D0B60E070E0CB010C94C70B6C
:1017B0000F931F9341E050E060E070E08A019B01CD
:1017C00004C0000F111F221F331F8A95D2F7C901D1
:1017D000B8011F910F910C94C70B0F931F9341E019
:1017E00050E060E070E004C0440F551F661F771F93
:1017F0008A95D2F78091320290913302A0913402FF
:10180000B09135028A019B01082B192B2A2B3B2B07
:10181000C901B8011F910F910C94C70B0F931F932F
:1018200041E050E060E070E004C0440F551F661FC7
:10183000771F8A95D2F74095509560957095809165
:10184000320290913302A0913402B09135028A01A4
:101850009B01082319232A233B23C901B8011F91A7
:101860000F910C94C70B0F931F9341E050E060E081
:1018700070E004C0440F551F661F771F8A95D2F78A
:101880008091320290913302A0913402B0913502DE
:101890008A019B01082719272A273B27C901B8017C
:1018A0001F910F910C94C70B0F931F93009132025D
:1018B000109133022091340230913502602B712B4C
:1018C000822B932B1F910F910C94C70B0F931F9397
:1018D000009132021091330220913402309135028E
:1018E00060237123822393231F910F910C94C70BC4
:1018F0000F931F9300913202109133022091340212
:101900003091350260277127822793271F910F910D
:101910000C94C70B08952FE0929F800D1124E82F9F
:10192000E695E695E695877051E001C0550F8A95DA
:10193000EAF785E0E89FF0011124E050FE4F20E037
:1019400030E070E04081CB01022E02C09695879571
:101950000A94E2F7817081958427852384278193F7
:101960002F5F3F4F2530310569F708952FE0929F93
:10197000800D1124682F669566956695982F97704F
:1019800085E0689FB001112440E050E080E0FB0159
:10199000E40FF51FE050FE4F208130E0092E02C019
:1019A000369527950A94E2F721703327042E01C05B
:1019B000220F0A94EAF7822B4F5F5F4F45305105A3
:1019C00031F70895BF92CF92DF92EF92FF920F937B
:1019D0001F93CF93DF938C01C0903202D0903302DB
:1019E000E0903402F09035028091360290913702F7
:1019F000A0913802B0913902C82AD92AEA2AFB2AD2
:101A0000CFE1D0E0D701C6010C2E04C0B695A79552
:101A1000979587950A94D2F780FD04C0219790F797
:101A2000B12C07C0BC2EB8018C2F0E943F14019727
:101A3000A9F38B2DDF91CF911F910F91FF90EF9024
:101A4000DF90CF90BF900895CF93DF93EC010E9479
:101A5000E20CBE010E943F14DF91CF9108951F93C5
:101A6000CF93DF93EB019091FF01992321F0CB01FC
:101A70000E94240D13C0882349F0CB010E94E20C80
:101A8000182F682FCE010E948B0C04C0CB010E943E
:101A9000B60C182FBE01812F0E943F14DF91CF9109
:101AA0001F9108951F93CF93DF93C0913A0216E0E0
:101AB00080913B02C81799F0D0E01C9FF0011D9F58
:101AC000F00D1124E45CFD4F4081518162817381EE
:101AD000848195810E946B0B2196C770E9CFDF91BD
:101AE000CF911F91089540916C0250916D026091C9
:101AF0006E0270916F0280917002909171020C944D
:101B00006B0BEF92FF920F931F93CF93DF93809114
:101B1000710282958F7009F065C080916E028823F2
:101B200009F460C080913A02F0903B0210916C027F
:101B300000916D0260916F027091700291E01F3F01
:101B400009F090E0C0910001D0910101292F96E0A9
:101B5000E92E8F1509F446C06115710521F00F3F7C
:101B600021F030E003C031E001C0322F90E030FDC1
:101B700036C0E89EF001E99EF00D1124DF01A45C5F
:101B8000BD4F11963C911197301329C03C913113F0
:101B900026C012963C911297311121C013964D9197
:101BA0005C911497461B570B4C175D07C0F480914E
:101BB00071028F70806180937102EF5BFD4F8081B5
:101BC0008F70806180838CE692E00E94E90ADF9149
:101BD000CF911F910F91FF90EF900C94520D0196B1
:101BE0008770B7CFDF91CF911F910F91FF90EF904A
:101BF00008959F92AF92BF92CF92DF92EF92FF92A1
:101C00000F931F93CF93DF93CDB7DEB761970FB6D6
:101C1000F894DEBF0FBECDBF8C0185E0F801DE0178
:101C20001D9601900D928A95E1F7D8011296EC90DD
:101C300090916C02E0916D0220916F0230917002E0
:101C40002115310531F0EF3F31F481E09F3F19F468
:101C500003C081E001C080E0B82FB1709B2E80FDF1
:101C600047C1D8014C9111965C9111971396AD9094
:101C7000BC9014978CE6C82E82E0D82EF0906E02AD
:101C8000B501621B730B2091000130910101FF200F
:101C900009F4D9C0809171026217730708F095C0EA
:101CA000282F207F09F052C05E1313C0491311C0C2
:101CB000FE2CE1100EC08F708061809371020E9433
:101CC000730DC6010E94E90A80917102F8018583B3
:101CD0004DC1AB2831F05F3F31F481E04F3F19F443
:101CE00003C081E001C080E080FD03C081E08E255B
:101CF00002C080E090E0F82FF170FF2E80FF1CC042
:101D000080913A0220913B0236E0821709F40BC120
:101D100090E0389FF001399FF00D1124E45CFD4FF5
:101D20006181561306C06081461303C06281E612CA
:101D300003C001968770E9CFFE2CEE2009F416C18E
:101D40008091710281608093710254C05E1306C05D
:101D5000491304C0E11002C0F80199C0C8010E94F3
:101D6000540B882361F1EE2051F120917102822FF2
:101D700082958F7090E0029774F080916C02909140
:101D80006D0298878F831986BB86AA862C87CE0121
:101D900007960E94E90A86E0F801ACE6B2E00190FD
:101DA0000D928A95E1F70E94810D0E94730D0AC081
:101DB0005E1711F1C8010E94540B81112CC0C8019B
:101DC0000E94E90AFF24F394D1C0282F207F81F7D5
:101DD0007A2DB98AA88A6E2D89890E945C0B8CE6BF
:101DE00092E00E94E90A86E0D6011D928A95E9F701
:101DF0000E94730DF12CBAC04913DCCFE110DACF89
:101E0000F8018583C8010E94E90A86E0D6011D9287
:101E10008A95E9F7ABC0EE2091F220917102822FF2
:101E200082958F7090E002970CF4B5CF80916C0290
:101E300090916D029A8389831B82BD82AC822E832E
:101E4000CE010196A6CF6217730708F044C0FE2C9E
:101E5000EE2009F4B4CF5E1330C049132EC0209198
:101E6000710220FD21C0822F82958F70482F50E093
:101E700041155105C9F0F80125834F30510541F056
:101E80008F5F982F9295907F822F8F70892B8583FB
:101E9000C8010E94E90A86E0F801ACE6B2E00190D0
:101EA0000D928A95E1F73CC086E0F801ACE6B2E01D
:101EB00001900D928A95E1F759C0C8010E94540B18
:101EC000811169CF80917102816080937102C80194
:101ED0000E94E90A4BC07A2DB98AA88A6E2D898999
:101EE0000E945C0B86E0D6011D928A95E9F718C026
:101EF000EE2009F464CFC8010E94540BF82E882309
:101F000009F45DCF86E0F801ACE6B2E001900D92F5
:101F10008A95E1F78CE692E00E94DD070E94810D30
:101F20000E94730D23C04D875E878D859E850E941C
:101F3000240D292F22952F70223028F49F7039F01C
:101F4000811105C00BC0243028F49F7049F4805ED5
:101F5000883020F0C8010E94E90A9F2CF92C06C0A5
:101F6000D80115969C91907F91F7F8CF8F2D6196AF
:101F70000FB6F894DEBF0FBECDBFDF91CF911F919A
:101F80000F91FF90EF90DF90CF90BF90AF909F9018
:101F900008951F93CF93DF93CDB7DEB72C970FB67D
:101FA000F894DEBF0FBECDBF4F83588769877A870D
:101FB0008B879C87CE0107960E94F90D8823D1F06C
:101FC0009F8188852A853B85232B31F08F3F31F413
:101FD00081E09F3F19F403C081E001C080E080FDF3
:101FE00047C04F81588569857A858B859C850E947D
:101FF0006B0B3EC086E0FE013796DE011196019024
:102000000D928A95E1F7FF81E8856A857B856115E8
:10201000710531F0EF3F31F481E0FF3F19F403C067
:1020200081E001C080E080FD23C020913B0230E0D0
:10203000C90101968770992740913A0250E08417B0
:102040009507F1F1F983EA837D836C8396E0929F93
:10205000D001939FB00D1124A45CBD4FFE013196B9
:1020600001900D929A95E1F780933B020E94520DE8
:1020700016E080913A0290913B02891771F1189F06
:10208000C0011124845C9D4F0E94F90D882329F121
:10209000E0913A021E9FF0011124E45CFD4F408163
:1020A000518162817381848195810E946B0B809143
:1020B0003A0290E001968770992780933A02D9CF2F
:1020C0000E94350B10923B0210923A02ECE6F2E0CD
:1020D00086E0DF011D928A95E9F72C960FB6F894F9
:1020E000DEBF0FBECDBFDF91CF911F9108958091CC
:1020F0007A02859585958595089580917A028770F5
:10210000089590917A02977081E009F480E0089533
:1021100080918502089590918502892B8093850294
:102120000895809590918502892380938502089572
:1021300010928502089590918402892B80938402E5
:102140000895809590918402892380938402089554
:1021500010928402089580917B02089508950C9452
:10216000AE100C94AF109091CC0292FD08C09091EB
:102170007B02981721F080937B020C94B110089594
:1021800080917B02882329F010927B0280E00C94DE
:10219000B1100895CF93DF93E0910201F091030114
:1021A000809185028083E0910201F091030190818A
:1021B00080918402892B808380917B02882381F027
:1021C000E0910201F09103019081892B808380913D
:1021D0000201909103010E94292081110E94C010E8
:1021E000C0910201D091030148E050E062E772E043
:1021F000CE010E943329892B69F088E0FE01A2E715
:10220000B2E001900D928A95E1F7CE01DF91CF9176
:102210000C94A61FDF91CF9108950C94AE1090916D
:10222000CC0292FD10C098E0899F90011124262BCA
:1022300020937A020E94ED0B80917A028595859514
:1022400085950C940D110C94ED0B10927A0280E0A0
:102250000C940D1120917A028095822380937A024A
:10226000982F977099F430E0482F082E000C550BEA
:102270002417350759F09091CC0292FD07C085953F
:10228000859585950E940E0C0C9425110895CF9389
:102290009091CC0292FB222720F92817F9F0C82F41
:1022A000892FC0FB82F98093CC028091CB02909160
:1022B000CC020E94A91182E00E942A11809198020A
:1022C00080FF0CC01F92CF9389E392E09F938F937E
:1022D0000E943C060F900F900F900F90CF910895A1
:1022E0008091CC0282FB882780F991E089270C94A9
:1022F000471181E00C94471180E00C9447116FEF77
:102300007FEF80E090E00C946C2980E090E00E94E8
:10231000482921E0893E9E4F09F020E0822F089550
:1023200082E090E00C94402983E090E00C944029F6
:10233000CF9384E090E00E944029C82F82E290E091
:102340000E9440292C2F30E0A901582BCA01CF91BF
:102350000895CF93C92F682F84E090E00E944E2902
:102360006C2F82E290E0CF910C944E29AB01BC011E
:102370008FE090E00C946029AB01BC0183E190E018
:102380000C94602960E070E0CB010C94BC1160E01B
:1023900070E0CB010E94B6110C94C21169EE7EEF81
:1023A00080E090E00E946C2960E082E090E00E9472
:1023B0004E2960E083E090E00E944E2910923602A0
:1023C00010923702109238021092390260E084E0D5
:1023D00090E00E944E2960E082E290E00E944E2947
:1023E00060E085E090E00E944E2960E086E090E0A9
:1023F0000E944E296FEF87E090E00E944E2940E056
:1024000050E0BA0188E090E00E94602960E08DE031
:1024100090E00E944E2940E050E0BA0188E190E04F
:102420000E94602960E087E190E00E944E2940E030
:1024300050E0BA018CE190E00E94602960E070E019
:1024400080E290E00E946C2940E050E0BA0188E10F
:1024500090E00E9460290C94C7110C94CE11682F53
:102460008EE090E00C944E290E941E21609394020D
:1024700070939502809396029093970260939002D6
:10248000709391028093920290939302089585B77E
:10249000806885BF85B7806885BF089581E008950D
:1024A0000C944E1208950C9452120C9452120C94E7
:1024B00055120C9452120C9459120C9452120E9400
:1024C000471283E493E20E94901F0E945D120C94D5
:1024D0005B120E9453120C9452120E9436150C94F7
:1024E00050070E9409210E9461160E946D120C94EF
:1024F00057125F926F927F928F929F92AF92BF928C
:10250000CF92DF92EF92FF920F931F93CF93DF93BF
:10251000CDB7DEB72A970FB6F894DEBF0FBECDBF9A
:102520000E947616C82E81110E94341236E8832E3E
:1025300032E0932E00E010E0502E802F0E945A15BA
:102540005C01F401619071904F0168267926611455
:102550007104B1F40F5F1F4F0530110569F78FEF5C
:1025600089838A831B820E9412218160782F9D8338
:102570008C8349815A816B818D810E9493073AC077
:102580008091980281FD0E946315D12CEE24E39482
:10259000F12CC3018E219F21892B29F10E94501219
:1025A0008823A9F0DE825F82AE20BF2081E0AB28C5
:1025B00009F480E088870E9412218160782F9A8731
:1025C00089874E815F8168858A850E949307000F05
:1025D000111FF801EA57FD4F80819181E826F92605
:1025E000F182E08207C0D394EE0CFF1CFFE0DF1203
:1025F000D0CFB0CF81E0C11001C080E02A960FB6E5
:10260000F894DEBF0FBECDBFDF91CF911F910F9128
:10261000FF90EF90DF90CF90BF90AF909F908F9002
:102620007F906F905F9008950E9479120E94FF182A
:102630000C946107CF93DF930E944414EC01811541
:1026400021E5920708F045C0811530E5930708F0B1
:1026500094C0883E910528F5803E910508F0F8C0A9
:10266000883A910570F4853A910508F07CC0813074
:10267000910509F475C008F4E8C0049708F0E8C0B3
:10268000E4C08F3B910508F0E0C0C85AD0E0CC0F01
:10269000DD1FC65BDE4F0990D881C02DCE0194644A
:1026A000D8C0811540E2940758F4811551E0950790
:1026B00008F0CEC08D3E910508F4C7C09065C9C032
:1026C000C11580E4D80708F4C0C0DF70CE01906A5D
:1026D000C0C0811525E59207A8F4811534E593075C
:1026E00008F095C0811543E5940708F07BC081157B
:1026F00052E5950708F061C0D82FCC27CE01816F35
:10270000906AA7C0C11589E5D807A0F4C11528E5CE
:10271000D20708F082C0C11536E5D30708F095C08E
:102720008C2F0E94D8148F7190E0D82FCC27CE0127
:1027300090628FC0C1154AE5D40708F474C0CE0179
:1027400090568115904208F080C08D2F8F710E94A5
:10275000D814DD27D0628F71AE01582BCA0179C021
:1027600081E090E076C0C55AD0E0C858DE4F88813D
:10277000C82FD0E0CE0190646CC074E09695879528
:102780007A95E1F7282F23703C2F337081E090E099
:1027900002C0880F991F3A95E2F79C68AC01522B52
:1027A0009A019C2F9F709695969550E2959FE00117
:1027B0001124C9018C2B9D2B4CC08370992721E0DB
:1027C00030E002C0220F331F8A95E2F79C2F9695C6
:1027D000969580E2989FE0011124C22BD32BCE0165
:1027E0009C6837C08370992721E030E002C0220F37
:1027F000331F8A95E2F79C2F9695969540E2949F19
:10280000E0011124C22BD32BCE019A6822C0D82F0D
:10281000CC27CE01846F906A1CC0DC2FCC27CE0160
:10282000806F906A16C08C2F8F700E94D81494E02D
:10283000D695C7959A95E1F7CF70D0E0DC2FCC27DD
:10284000D0699E01282BC90104C080E090E001C03E
:10285000CE01DF91CF9108952BE4829FC001112416
:10286000FC012FE0729FE00DF11D1124E60FF11D18
:10287000EE0FFF1FE852FF4F8591949108950E943B
:102880002C140E941A1308958238910569F1B0F44E
:102890008133910509F46DC048F48932910509F43A
:1028A00063C08A32910509F469C0089585339105A2
:1028B00009F455C089339105B9F00895833E910517
:1028C00069F138F4803E9105B1F0823E910509F13D
:1028D0000895863E9105A9F1873E9105B9F1843EA0
:1028E000910509F064C023C02091CB0220FD4FC0A8
:1028F00021FD4DC008958091CB0280FD44C08091A0
:10290000CC0280FF44C08091CB0284FD42C083EEA4
:102910004DC08091CB0282FF38C0F5CF8091CB02B1
:1029200082FD33C08091CC0280FD31C0ECCF80911C
:10293000CC0281FF32C08091CB0284FD2AC087EE99
:1029400035C08091CB0283FF26C0F5CF8091CB02AA
:1029500083FD21C08091CC0281FD1FC0ECCF80910E
:10296000CB0285FD1CC01DC08091CB0285FD19C026
:1029700016C08091CB0286FD16C017C08091CB0295
:1029800086FD13C010C089E311C082EE0FC080EE37
:102990000DC080E00BC086EE09C084EE07C089E25E
:1029A00005C085E303C08AE201C081E390E0089599
:1029B0009091CB0292FF0DC0282F2871283019F476
:1029C000877F846006C0282F2471243011F48B7F08
:1029D000886093FF0DC0282F2871283119F4877E55
:1029E000846106C0282F2471243111F48B7E886104
:1029F0002091CC0220FF0DC0382F3871383019F4E7
:102A0000877F816006C0382F3171313011F48E7F9D
:102A1000886021FF0DC0282F2871283119F4877E86
:102A2000816106C0282F2171213111F48E7E8861C9
:102A300094FD877E08950C947F110E9476162FEFE7
:102A400086E791E0215080409040E1F700C000000F
:102A50000E94761680E00E945A1580FF04C00E94F2
:102A60001B150C945F2108950C941D150E9485116F
:102A7000811102C00E942D120E9490118093980231
:102A80000E9498119093CC028093CB020E9434153F
:102A90000E949411682F70E080E090E00E948D0BFE
:102AA000609132027091330280913402909135022C
:102AB0000C94C50BE82FF0E0EE0FFF1FE952FD4F1D
:102AC000808191810895CF92DF92EF92FF920F93D0
:102AD0001F93CF93DF938EE592E00E94A30587EDCD
:102AE000E82E82E0F82EC0E0D0E099E5C92E92E011
:102AF000D92E00E512E0DF93CF93DF92CF920E94B0
:102B00003C0686E592E00E94A305F7018191919130
:102B10007F010E9436079F938F931F930F930E940C
:102B20003C068EE492E00E94A30521968DB79EB7E5
:102B300008960FB6F8949EBF0FBE8DBFC530D10565
:102B4000D1F6DF91CF911F910F91FF90EF90DF9021
:102B5000CF90089580EA8A95F1F7089500C008950E
:102B60000C94AA1508950C94B2150C94B3150C94FA
:102B7000B2150C94B715F894E82FE295EF70F0E0D9
:102B800031A1282F2F7081E090E001C0880F2A9595
:102B9000EAF7982F9095932391A392A1892B82A372
:102BA000789408950F931F93CF93DF93CAE8D1E0F1
:102BB00089918F3F11F00E94BB1581E0CF38D80773
:102BC000B9F7CBE7D1E00AE811E089918F3F11F026
:102BD0000E94BB150C171D07C1F7DF91CF911F9104
:102BE0000F910895BF92CF92DF92EF92FF920F93D1
:102BF0001F93CF93DF938C01C62FD0E0CE01865771
:102C00009E4F6C01FC0190819F3F09F450C0B62E8D
:102C1000F894E92FE295EF70F0E081A19F7021E038
:102C200030E001C0220F9A95EAF7822B81A382A19E
:102C30002095282322A378940E94AE15EBE7F1E0BB
:102C40004AE851E021E030E0E12CF12C61916F3F46
:102C500089F0A62FA295AF70B0E090968C9190E08D
:102C60006F7002C0959587956A95E2F780FD02C066
:102C7000C90102C080E090E0E82AF92A220F331F40
:102C80004E175F0719F7F60180818F3F11F00E9400
:102C9000BB1561E0E114F10409F460E08B2D0E94A2
:102CA000B015CC0FDD1FC00FD11FF982E882DF9174
:102CB000CF911F910F91FF90EF90DF90CF90BF9039
:102CC00008950E94D2158AE0E7EDF2E0DF01982F27
:102CD0001D929A95E9F7EDECF2E0DF011D928A95DD
:102CE000E9F785E00E94C1160C949706FF920F93B6
:102CF0001F93CF93DF93CDB7DEB72A970FB6F89423
:102D0000DEBF0FBECDBF8E010F5F1F4F8AE0F801FF
:102D100011928A95E9F7F12C6F2DC8010E94F215E6
:102D2000F394F5E0FF12F8CF4AE050E0B8018DECE3
:102D300092E00E943329FF24F394009709F4F12CC8
:102D4000892B41F08AE0F801ADECB2E001900D92E0
:102D50008A95E1F72F2D45E067ED72E08DEC92E06A
:102D60000E94C2160E9499068F2D2A960FB6F894DB
:102D7000DEBF0FBECDBFDF91CF911F910F91FF90AE
:102D800008950895FF920F931F93CF93DF93F82E2A
:102D9000092F162FD72FC42F222349F081E08093CB
:102DA0009B020E94122190939A0280939902809133
:102DB0009B028823D9F08091990290919A020E94F7
:102DC0002A21059798F0EF2DF02FA12FBD2F80E03D
:102DD00090E04C2F50E08417950734F42191319105
:102DE0002D933D930196F7CF10929B02DF91CF91E7
:102DF0001F910F91FF9008950E94BF230E947112AE
:102E00000C94CB230E94CF230E9414130C94ED2327
:102E10000E94B0200E94A6230E945F120E94FC160E
:102E20000E9402170E946912FBCF8091A20280FFCC
:102E300006C06091090170E0660F771F26C081FF10
:102E400004C06091090184E005C082FF07C0609161
:102E5000090188E0689FB001112417C09091A10278
:102E60009923D1F060910801961788F72091090104
:102E700088E0289F90011124929FA001939F500DFC
:102E8000112470E0CA010E9405296038710540F4E0
:102E90006115710519F406C068E070E0862F089589
:102EA0008FE7089581E008958091A20280FF08C015
:102EB0006091050170E0759567957595679521C0DE
:102EC00081FF06C06091050170E07595679519C096
:102ED00082FF04C06091050170E010C09091A002D3
:102EE000992399F0609104019617A0F7809105014C
:102EF000899FC001112470E00E9405296038710586
:102F000040F46115710519F406C061E070E0862F88
:102F100008958FE7089581E008958D3E21F40E9481
:102F20001517819504C08E3E29F40E9415178093D1
:102F3000A60208958F3E21F40E941517819504C0C2
:102F4000803F29F40E9415178093A5020895893FB8
:102F500019F40E94541705C08A3F31F40E94541797
:102F600081958093A70208958B3F21F40E94541706
:102F7000819504C08C3F29F40E9454178093A802C5
:102F800008959FE0980F983078F421E030E0A9018F
:102F900002C0440F551F9A95E2F7CA019091A4020E
:102FA000892B8093A40208958D3F21F48091A20281
:102FB00081600BC08E3F21F48091A202826005C027
:102FC0008F3F29F48091A20284608093A202089529
:102FD0008D3E39F49091A60297FF35C01092A6025B
:102FE00059C08E3E29F49091A6021916BCF32BC04D
:102FF0009091A5028F3E29F497FF25C01092A5025B
:1030000049C0803F19F41916CCF31DC09091A70256
:10301000893F29F41916BCF41092A7023BC08A3FDD
:1030200019F497FF10C0F8CF8B3F39F49091A802A4
:1030300097FF09C01092A8022DC08C3F21F49091F7
:10304000A8021916BCF39FE0980F983080F421E095
:1030500030E0A90102C0440F551F9A95E2F7CA015A
:1030600080959091A40289238093A40213C08D3F80
:1030700021F48091A2028E7F0BC08E3F21F48091BB
:10308000A2028D7F05C08F3F29F48091A2028B7F21
:103090008093A2028091A502811106C08091A602B0
:1030A000811102C01092A1028091A702811106C075
:1030B0008091A802811102C01092A002089580910F
:1030C000980283FF7EC08CE992E00E94A305809164
:1030D000A4021F928F9387E992E09F938F930E949F
:1030E0003C0685E992E00E94A3058091A502282F65
:1030F000082E000C330B3F938F9382E992E09F934D
:103100008F930E943C0680E992E00E94A305809183
:10311000A602282F082E000C330B3F938F938DE8C7
:1031200092E09F938F930E943C068BE892E00E946E
:10313000A3058091A702282F082E000C330B3F9384
:103140008F9388E892E09F938F930E943C0686E8D5
:1031500092E00E94A3058091A802282F082E000C5F
:10316000330B3F938F9383E892E09F938F930E945A
:103170003C0680E892E00E94A3058091A1021F9284
:103180008F938DE792E09F938F930E943C068BE78D
:1031900092E00E94A3058091A2021F928F9388E77C
:1031A00092E09F938F930E943C0685E792E00E94F5
:1031B000A3058DB79EB74C960FB6F8949EBF0FBE71
:1031C0008DBF0E9412212091A502211104C02091DF
:1031D000A602222321F090939F0280939E022091C9
:1031E000A702211104C02091A802222321F090936C
:1031F0009D0280939C0283EA92E00C94EF1FEF9271
:10320000FF920F931F93CF93DF9300D000D000D095
:10321000CDB7DEB786E0E3EAF2E0DE011196019079
:103220000D928A95E1F7E090A502F090A602009138
:10323000A7021091A8021092A5021092A602109265
:10324000A7021092A802E11003C0FF2009F45DC09C
:1032500080919E0290919F020E942A21AC01909140
:10326000A102992339F020910A0130E02417350793
:1032700058F04BC020910B018AE0289F9001112447
:103280002417350718F041C09F3F19F09F5F9093B6
:10329000A102EE2061F00E9415171E1414F09FEF9A
:1032A00001C091E0989F902D11249093A502FF20DA
:1032B00061F00E9415171F1414F09FEF01C091E0F8
:1032C000989F902D11249093A6023091A50233234C
:1032D000E1F02091A6022223C1F045EB3403C001A6
:1032E0001124992319F09093A50203C081E08093E3
:1032F000A50235EB2303C0011124992319F0909303
:10330000A60203C081E08093A602011103C011232D
:1033100009F45DC080919C0290919D020E942A2137
:10332000AC019091A002992339F02091060130E080
:103330002417350758F04BC0209107018AE0289FD9
:10334000900111242417350718F041C09F3F19F050
:103350009F5F9093A002002361F00E945417101603
:1033600014F09FEF01C091E0989F902D112490934D
:10337000A702112361F00E945417111614F09FEF59
:1033800001C091E0989F902D11249093A802309154
:10339000A7023323E1F02091A8022223C1F045EBDC
:1033A0003403C0011124992319F09093A70203C09C
:1033B00081E08093A70235EB2303C00111249923F8
:1033C00019F09093A80203C081E08093A802809135
:1033D000A50281110BC08091A602811107C08091C6
:1033E000A702811103C08091A80281110E945F1879
:1033F000EB82FC820D831E8386E0FE013196A3EAF8
:10340000B2E001900D928A95E1F726960FB6F894F6
:10341000DEBF0FBECDBFDF91CF911F910F91FF9007
:10342000EF900895E3EAF2E086E0DF011D928A95CD
:10343000E9F71092A1021092A0021092A202089540
:10344000CF93DF93EC01FB018281882309F43CC117
:10345000C430FDE5DF0760F4CB3F9CE5D90788F475
:103460009E0122503C452431310508F02EC109C08F
:10347000C236EDE5DE0729F0C63AFDE5DF0709F0C3
:1034800024C10E9498119093CC028093CB02C13149
:103490008CE5D80709F4C6C008F042C0C930ECE595
:1034A000DE0709F49BC000F5C5308CE5D80709F4A8
:1034B00085C078F4C330ECE5DE0709F478C008F085
:1034C0007AC0C230DC4509F0F5C08091CB02816042
:1034D000EFC0C7309CE5D90709F478C008F07AC07E
:1034E0008091CB028061E4C0CD30FCE5DF0709F4B8
:1034F00087C058F4CB309CE5D90709F479C008F0AF
:103500007BC08091CB0288606FC0CF30FCE5DF07C5
:1035100009F480C008F082C08091CB02877FC8C0C8
:10352000CE3F9CE5D90709F471C000F5C531FCE533
:10353000DF0709F485C068F4C3319CE5D90709F4B5
:1035400075C008F095C00E94350B8091CB028F7733
:10355000AFC0CC3FFCE5DF07A9F108F054C0CB3F7A
:10356000DC4509F0A7C08091CC0240C0C230EDE537
:10357000DE0709F489C058F4C1158DE5D80709F4B0
:103580005AC008F069C08091CC0282602FC0C23658
:10359000EDE5DE0709F47CC0C63AFDE5DF0709F476
:1035A00081C0C330DD4509F085C080E06EC08091E8
:1035B000CB0282607DC08091CB0216C08091CB028D
:1035C000886076C08091CC0282604FC08091CB022F
:1035D00080626EC08091CB0280646AC00E94350B0D
:1035E0008091CB02806864C0846062C081603DC00D
:1035F0008091CB028E7F5CC08091CB028D7F58C0C2
:103600008091CB0216C08091CC0218C08091CC0270
:103610008D7F2BC08091CB028F7E4AC08091CB02E0
:103620008F7D46C08091CB028F7B42C08091CB02C0
:10363000877F8B7F3DC08091CC028D7F8E7F15C0B0
:103640008091CB0282FB222720F991E0922790FB08
:1036500082F990FB83F92CC08091CC02982F909531
:1036600091708E7F892B90FB81F98093CC0222C0D0
:103670000E94350B8091CB0287FB222720F991E035
:10368000922790FB87F914C081E00E942F1212C08C
:103690008091CB0284FB222720F991E0922790FBB6
:1036A00084F906C08091CB02982F909590FB80F909
:1036B0008093CB028091CB029091CC020E94A91101
:1036C0000E94350B80E001C081E0DF91CF91089529
:1036D000809104011F928F93809105011F928F9317
:1036E000809108011F928F93809109011F928F93FF
:1036F00080910A011F928F9380910B011F928F93EB
:103700008FEB92E09F938F930E943C068DB79EB7FC
:103710000E960FB6F8949EBF0FBE8DBF08958832E7
:1037200020F58E3108F068C08B3091F1C0F48730FD
:1037300009F0BEC081E080930B0184E180930A010F
:103740008AE0809309018EE18093080188E08093EC
:10375000050188E28093040181E294E0C6C08331D0
:1037600009F443C0843169F1A3C08F3409F49EC0C9
:1037700028F4893231F1883359F09AC0813531F01B
:1037800008F4D4C0823509F4A7C092C08FEFA5C059
:1037900083E494E00E94A3050E94681B1F9281E0CD
:1037A0008F931F9288E08F938CE393E09F938F9386
:1037B0000E943C060F900F900F900F900F900F906B
:1037C00096C080E494E00E94A3058091AD02882316
:1037D00009F4AAC01092AD021092AC021092AB0292
:1037E0001092AA021092A902B1C082E394E00E9452
:1037F000A3050E94681B7BC08D518093AD0283306E
:1038000031F170F48130D1F0823009F03FC08AE0AC
:1038100091E09093AC028093AB028CE991E01FC0E1
:10382000853059F108F1863089F584E091E0909374
:10383000AC028093AB0287ED91E011C08BE091E088
:103840009093AC028093AB0283E991E008C089E0D9
:1038500091E09093AC028093AB0288EA91E0909360
:10386000AA028093A90218C088E091E09093AC026C
:103870008093AB0285EB91E0F2CF85E091E09093ED
:10388000AC028093AB0284EC91E0E9CF1092AD02E0
:103890008FE294E00E94A3058091AD02882309F491
:1038A00055C01F928F938BE294E00DC08AE015C043
:1038B0008EE194E01AC097FF47C0108280811F926A
:1038C0008F9388E194E09F938F930E943C060F9022
:1038D0000F900F900F900BC081E0E091AB02F09140
:1038E000AC02309729F585E194E00E94A305209170
:1038F000AD02222359F18091A9029091AA0200976A
:1039000011F48FE891E09F938F931F922F938CE097
:1039100094E09F938F930E943C060F900F900F901E
:103920000F900F900F9016C080E0089586EFD5CFCE
:103930002081082E000C990B820F911D8F3F91055D
:1039400009F00CF4B8CF8FEF8083B8CF88E094E013
:103950000E94A30581E00895CF93C82F1F928F93F3
:1039600089E594E09F938F930E943C0681E090E06C
:10397000A0E0B0E0BC01CD0104C0660F771F881F36
:10398000991FCA95D2F70E948D0B0F900F900F9040
:103990000F90CF910C94350BEF92FF920F931F93E2
:1039A000CF93DF938B3109F4EDC008F08EC08B30DC
:1039B00009F4B1C008F078C0863009F4AFC020F433
:1039C000853009F4BDC04EC1873009F4C0C08830CD
:1039D00009F048C10E9494111F928F9382E898E0E9
:1039E0009F938F930E943C060E94901183FB99271E
:1039F00090F91F929F9382FB992790F91F929F93B2
:103A000081FB992790F91F929F93982F91701F9295
:103A10009F931F928F9389E398E09F938F930E94C7
:103A20003C060E94981187FB222720F91F922F93B2
:103A300086FB222720F91F922F9385FB222720F94E
:103A40001F922F9384FB222720F91F922F9383FB31
:103A5000222720F91F922F9382FB222720F91F9201
:103A60002F9391FB222720F91F922F93292F21704A
:103A70001F922F9381FB222720F91F922F93282F2B
:103A800021701F922F939F938F9384E597E09F93CC
:103A90008F930E943C068DB79EB788960FB6F89418
:103AA0009EBF0FBE8DBF35C0803109F495C020F494
:103AB0008E3009F47BC0D6C0863109F4A8C08931A4
:103AC00009F0D0C089EC94E084C08A32E1F060F45F
:103AD000873209F4C3C028F48E3108F4C3C08D5175
:103AE000BEC0893269F1BEC0833448F48A3308F01D
:103AF000B3C0853309F4B2C0883369F0B3C08334EE
:103B000009F4ACC0AFC08DE299E00E94A3050E9409
:103B10002D12C1E0ACC081EB95E05BC080919802B2
:103B2000817F8E7F809398028AE895E00E94A305AA
:103B300089E299E00E94A30581E08093AE02E9CF7B
:103B40008DE099E00E94A3050E949C06E2CF80913F
:103B50009802C82FC095C170C0FB80F9809398026D
:103B6000CC2329F081E099E00E94A30580C084EF76
:103B700098E00E94A30580919802897F877F8093B7
:103B80009802C7CF9091980291FBCC27C0F981E0B1
:103B9000C827892FC0FB81F980939802CC2319F0A4
:103BA00087EE98E029C089ED98E013C090919802C3
:103BB00092FBCC27C0F981E0C827892FC0FB82F98E
:103BC00080939802CC2319F08AEC98E015C08AEB18
:103BD00098E00E94A3059DCF9091980293FBCC277B
:103BE000C0F981E0C827892FC0FB83F98093980230
:103BF000CC2351F08EEA98E00E94A30580919802B0
:103C000081608093980233C081EA98E0E2CF0E94FD
:103C10001E21162F072FF82EE92ED091CA02C0912F
:103C200018010E949A1FEF92FF920F931F931F9209
:103C3000DF931F92CF931F928F938EE594E09F9313
:103C40008F930E943C068DB79EB70C960FB6F894E2
:103C50009EBF0FBE8DBF5DCF895301C080E00E9423
:103C6000AC1C57CF8FE998E00E94A305C0E08C2FD1
:103C7000DF91CF911F910F91FF90EF90089580E019
:103C800008950C943F1ECF93C82F8091AE028130CF
:103C900071F040F0823009F045C08C2F0E948F1BDC
:103CA00081E046C00E9488108232F1F504C00E9473
:103CB0008810823261F48C2F0E94411E811104C051
:103CC0008C2F0E94CC1C2CC081E090E029C08C2F4E
:103CD0000E943F1E811123C0C431C9F058F4CB307B
:103CE00069F0C031B9F482E08093AE0288E30E94AB
:103CF0008F1B15C0C93259F0C83361F48AE895E0CA
:103D00000E94A30585E594E00E94A30508C01092D7
:103D1000AE020CC083E594E00E94A30507C081E0D9
:103D2000817006C01092AE0280E002C080E0F8CF41
:103D3000CF910895CF93DF9386319C4541F5EB01F8
:103D40000E948810982F8A812091020130910301EE
:103D5000882379F09A7A81E009F480E08093AF02B9
:103D6000911102C069E201C065E3C9010E946B20A4
:103D70000AC08091AF02811102C069E201C065E30F
:103D8000C9010E946D200E94CA1080E001C081E03C
:103D9000DF91CF9108950F931F93CF93DF93C42F9B
:103DA000D22FFC0182818823C9F04093B2020E9485
:103DB00012219093B1028093B00280E28C0F883080
:103DC00008F057C0C77081E001C0880FCA95EAF7B4
:103DD000DF91CF911F910F910C9492088091B202C4
:103DE000481330C08091B0029091B1020E942A2104
:103DF000883C910538F510E21D0FCD17B9F080E22F
:103E00008C0F883040F4C77081E001C0880FCA95DC
:103E1000EAF70E949908183028F581E09D2F9770E5
:103E200001C0880F9A95EAF70E949208802F0E949D
:103E300089081830F0F4D77081E001C0880FDA9556
:103E4000EAF70AC080E28C0F883098F4C77081E0EE
:103E500001C0880FCA95EAF7DF91CF911F910F91AA
:103E60000C949908802FDF91CF911F910F910C94A2
:103E70008908DF91CF911F910F9108950F939C01B5
:103E8000CB01243F4CE5340731F188F4293DFCE5B2
:103E90003F07D9F02A3D4CE5340779F1283D3C45F0
:103EA000A9F506E221EE41EE68ED7CE52BC0263F48
:103EB000FCE53F07E1F0A8F0273F3C4539F507E274
:103EC00025EE46EE67EF7CE51DC007E225EE45EEE8
:103ED00069ED7CE517C006E221EE40EE64EF7CE57B
:103EE00011C007E225EE44EE65EF7CE50BC006E26B
:103EF00021EE42EE66EF7CE505C008E221E045EEEA
:103F00006AED7CE50E94CB1E80E008C0FC01828146
:103F1000882319F01092B20201C081E00F91089538
:103F20009093FD018093FC0108959093B8028093D3
:103F3000B7020895E091B702F091B802309721F0EE
:103F40000190F081E02D099480E00895EF92FF92B6
:103F50000F931F93CF93DF93E091B702F091B802D4
:103F60003097B1F18C010280F381E02D09958091A9
:103F7000980282FF2DC080FF04C086E499E00E9471
:103F8000A305E80118E080E4E82E89E0F82E80918E
:103F9000980280FF0BC088811F928F93FF92EF924F
:103FA0000E943C060F900F900F900F901150219699
:103FB0001111EDCF8091980280FF0AC08EE399E045
:103FC000DF91CF911F910F91FF90EF900C94A3057B
:103FD000DF91CF911F910F91FF90EF900895E091A5
:103FE000B702F091B802309739F022E0DC012C934F
:103FF0000480F581E02D099408952091B502309157
:10400000B6022817390771F09093B6028093B50273
:10401000E091B702F091B802309721F00680F78165
:10402000E02D099408952091B3023091B40228172D
:10403000390771F09093B4028093B302E091B70214
:10404000F091B802309721F00084F185E02D0994B9
:104050000895FC01329697E080E0915029F021917B
:104060002223D9F38F5FF9CF0895662349F0FC012D
:10407000329608962191621729F0E817F907D1F7CF
:1040800080E0089581E008959C01FC0132969FEF45
:1040900080E04191461789F09F3F19F4411101C01A
:1040A000982F8F5F8630A9F79F3F39F0F901E90F0C
:1040B000F11D97FDFA956283089508959C012A5F8A
:1040C0003F4FFC014281461301C0128201968217C4
:1040D0009307B9F708950C9444200C945E2002963F
:1040E00026E0FC0111922A95E9F7089508950C94B1
:1040F000762083E08093B9020C947720811102C06E
:1041000081E001C082E08093B9020C9477200C9486
:104110007E2081E08093B9020C9477200C94892052
:1041200008950C9490200C9491200C9490200C9461
:1041300090200C949020CF930E9497200E94761696
:104140000E949520C0E08C2F0E945A15892B29F4DB
:10415000CF5FC530C1F780E001C081E0CF91089505
:1041600008951F920F920FB60F9211248F939F9371
:10417000AF93BF938091BA02811113C08091E10285
:104180009091E202A091E302B091E4024196A11D58
:10419000B11D8093E1029093E202A093E302B093F9
:1041A000E402BF91AF919F918F910F900FBE0F903E
:1041B0001F9018958091E902843031F10E941C070C
:1041C0001092BA0220E488E190E00FB6F894A89526
:1041D000809360000FBE2093600083B7817F84606E
:1041E00083BF83B7816083BF7894889583B78E7FC0
:1041F00083BF0FB6F894A895809160008861809382
:104200006000109260000FBE08950E94350B0C9460
:10421000200782E084BD93E095BD9AEF97BD80931F
:104220006E0008952FB7F8948091E1029091E20218
:10423000A091E302B091E4022FBF08952FB7F89444
:104240006091E1027091E2028091E3029091E402B8
:104250002FBF08959C014FB7F8948091E10290918F
:10426000E202A091E302B091E4024FBF821B930BE4
:10427000089578941F920F920FB60F9211248F9386
:104280009F93AF93BF938091E1029091E202A0913E
:10429000E302B091E4020196A11DB11D8093E102F9
:1042A0009093E202A093E302B093E402BF91AF9136
:1042B0009F918F910F900FBE0F901F90189587E7D9
:1042C00097E790930108809300089AE088E10FB681
:1042D000F894A895809360000FBE90936000FFCF84
:1042E0008091C9020895089522E02093E9002FEFFC
:1042F0003091E800215035FD06C035ED3A95F1F7D3
:1043000000002111F5CF2091E80025FF0BC040E00F
:1043100050E066E070E00E945C248091E8008E77B7
:104320008093E8000895CF93DF9321E02093E90084
:104330002FEF3091E800215035FD06C035ED3A955C
:10434000F1F700002111F5CF2091E80025FF14C0FE
:10435000EC0140E050E068E070E00E945C24809155
:10436000E8008E778093E80088E0FE01A1ECB2E0DF
:1043700001900D928A95E1F7DF91CF910895809396
:10438000BD027093BF026093BE028091E902843047
:1043900001F582E08093E9008FEF9091E800815071
:1043A00095FD06C095ED9A95F1F700008111F5CFC6
:1043B0008091E80085FF0DC040E050E063E070E0D0
:1043C0008DEB92E00E945C248091E8008E778093D0
:1043D000E8000895BC0184E00C94BF21BC0183E097
:1043E0000C94BF218CE699E00E94A3058091E8021D
:1043F000811109C00E94ED250E944A268091E200A9
:1044000084608093E200089588E699E00E94A30505
:104410001092E802089584E699E00E94A3050C94A6
:104420008E2080E699E00E94A3056091E50281E07C
:10443000611101C080E00C9479208CE599E00E9424
:10444000A3059091E90281E0943009F080E0609149
:10445000E5020C947E202091BC022F5F822F62E344
:104460000E94F928992319F02093BC020895109214
:10447000BC028091C002882371F18091E9028430EE
:1044800041F58091E9008F702091EC00922F91709E
:1044900020FD90E8892B93E09093E9009091EB0048
:1044A00090FF14C09091EE0097FF10C09091E8002B
:1044B00095FF03C01092F100F9CF9091E80090FFB2
:1044C00005C09091E8009E779093E8008F708093EC
:1044D000E9001092C002089542E061EC81E00E9480
:1044E000662542E261EC82E00E94662542E261ECD0
:1044F00083E00E9466259091E90281E0943009F002
:1045000080E06091E5020C9487208091EB0283307B
:1045100009F461C030F4813071F0823009F49AC03E
:1045200008958A3009F486C08B3009F46CC0893054
:1045300009F0A8C020C08091EA02813A09F0A2C027
:104540008091E800877F8093E8008091EE0290914F
:10455000EF02892B21F468E081EC92E003C060E077
:1045600080E090E070E00E94A7248091E8008B77C3
:104570008093E80008958091EA02813209F082C0B8
:104580008091EE029091EF02029708F07BC080913B
:10459000E800877F8093E8008091E80082FD05C0F5
:1045A0008091E9028111F8CF6DC02091F3008091D4
:1045B000F20090E0922B029731F48091F10081306B
:1045C00011F0863021F48091F1008093C90280912E
:1045D000E8008B7753C08091EA02813A09F052C01B
:1045E0008091EE029091EF02892B09F04BC08091EF
:1045F000E800877F8093E8008091E80080FFFCCF8F
:104600008091180136C08091EA028132D9F58091FB
:10461000EE029091EF02892BA9F58091E800877F47
:104620008093E8000E949B258091EC028093180102
:104630000C94350B8091EA02813221F58091E800DB
:10464000877F8093E8000E949B258091ED028093F4
:10465000CA0208958091EA02813AA1F48091E800AB
:10466000877F8093E8008091E80080FFFCCF8091F5
:10467000CA028093F1008091E8008E778093E80071
:104680000C949B2508959FB7F8941092C0029FBF89
:104690009091E902943009F057C09091E9009F7021
:1046A0003091EC00232F217030FD20E8922B23E085
:1046B0002093E9002091EB0020FF43C02091EE0001
:1046C00027FF3FC02091BB02222321F02091E80068
:1046D00025FF37C01092BB0226E03091E80035FD7F
:1046E00015C03091E902343061F53091EB0035FDB1
:1046F00028C0215021F481E08093BB0222C0EFE961
:10470000FFE03197F1F700C00000E7CF8093F100A0
:104710008091E80085FD0AC08091E80080FFFCCF11
:104720008091E8008E778093E80006C08FB7F894F8
:1047300021E02093C0028FBF9F709093E90080E03A
:1047400008959F709093E9008FEF089584B7877F55
:1047500084BF0FB6F894A89580916000886180931B
:104760006000109260000FBE90E080E80FB6F894F1
:1047700080936100909361000FBE0C9489200E9489
:10478000ED250E944A26E2EEF0E08081846080837D
:1047900078940C94DE288CE091E00C94951F809125
:1047A000E9028530C9F488E599E00E94A30580916B
:1047B000E902853079F40E94DA208091E7028823AB
:1047C000B1F30E949B20882391F30E9446240E940B
:1047D000350BEDCF0C940521089508950C94F0232A
:1047E000292F332723303105C9F060F421303105FA
:1047F00081F02230310509F041C08BE590E026EAD6
:1048000039E040C021323105E1F02232310531F189
:1048100035C082E190E021E03AE034C09927813050
:10482000910549F028F0029749F5E0E7F9E005C065
:10483000E2EAF9E002C0E6E8F9E0849190E09F0145
:1048400021C063307105D0F4660F771FFB01EB5078
:10485000FE4F2081318189E090E014C06330710502
:1048600068F4FB01EE0FFF1FE151FE4F2081318103
:10487000FB01E451FE4F808190E004C080E090E0B5
:1048800020E030E0FA0131832083089580E189BD82
:1048900082E189BD09B400FEFDCF8091D8008F7DF3
:1048A0008093D8008091E00082608093E000809146
:1048B000E00081FDFCCF0895CF92DF92EF92FF924E
:1048C0000F931F93CF93DF93EC018B017A010E942A
:1048D000BA25811133C0E114F10439F0F701808168
:1048E0009181081B190BC80FD91FC12CD12C0115A0
:1048F000110519F18091E80085FD16C08091E8004E
:104900008E778093E800E114F10449F0F70180818B
:104910009181C80ED91ED182C08285E00FC00E944D
:10492000BA25882321F30AC089918093F1000150B0
:104930001109FFEFCF1ADF0ADACF80E0DF91CF91C4
:104940001F910F91FF90EF90DF90CF9008952091ED
:10495000F0023091F1022617370748F06115710512
:1049600039F42091E8002E772093E80001C0B901C6
:10497000FC0120E06115710579F18091E90288233D
:10498000F1F18530F1F18091E80083FD3CC0809128
:10499000E80082FD2EC08091E80080FFEBCF2091DF
:1049A000F3008091F20090E0922B6115710551F0B7
:1049B0008830910538F421912093F10061507109FC
:1049C0000196F3CF21E0089709F020E08091E800FC
:1049D0008E778093E800CECF2111CFCF0AC080918F
:1049E000E902882361F0853061F08091E80083FD61
:1049F0000AC08091E80082FFF2CF80E0089582E053
:104A0000089583E0089581E008952091F0023091A7
:104A1000F1022617370748F06115710539F4209126
:104A2000E8002E772093E80001C0B901FC0120E0E6
:104A30006115710591F18091E902882309F440C064
:104A4000853009F43FC08091E80083FD3DC080912E
:104A5000E80082FD2FC08091E80080FFE9CF20911F
:104A6000F3008091F20090E0922B6115710559F0EE
:104A70008830910540F424912093F10031966150E3
:104A800071090196F2CF21E0089709F020E08091AA
:104A9000E8008E778093E800CBCF2111CCCF0AC0FD
:104AA0008091E902882361F0853061F08091E8000F
:104AB00083FD0AC08091E80082FFF2CF80E0089574
:104AC00082E0089583E0089581E00895982F97305B
:104AD00068F59093E900981739F07091EC002091F7
:104AE000ED005091F00003C0242F762F50E021FDFF
:104AF00002C09F5FECCF3091EB003E7F3093EB0024
:104B00003091ED003D7F3093ED003091EB0031604E
:104B10003093EB007093EC002093ED005093F00085
:104B20002091EE0027FDE5CF80E008958F708093FF
:104B3000E90081E008958091EA0287FF11C0809129
:104B4000E80082FD05C08091E9028111F8CF11C013
:104B50008091E8008B770BC08091E902882349F0AF
:104B60008091E80080FFF8CF8091E8008E778093F5
:104B7000E80008952091E4003091E50095E6409129
:104B8000EC00842F817040FF23C08091E80080FDFD
:104B90001DC08091E902882399F0853099F08091B9
:104BA000EB0085FD11C04091E4005091E500241711
:104BB000350729F3915011F09A01E1CF84E008956F
:104BC00082E0089583E0089581E0089580E00895EB
:104BD0004091E80042FFDDCF08950E945B260E94CD
:104BE0006326E0EEF0E0808181608083E8EDF0E014
:104BF00080818F77808319BCA7EDB0E08C918E7F88
:104C00008C9380818F7E80831092E80208950F93A9
:104C10001F93CF93DF930E945B260E946326C8ED0B
:104C2000D0E088818F7788838881806888838881B5
:104C30008F7D888319BC1092E9021092E5021092D0
:104C4000E7021092E60200EE10E0F80180818B7F0F
:104C5000808388818160888342E060E080E00E94F8
:104C60006625E1EEF0E080818E7F8083E2EEF0E069
:104C7000808181608083808188608083F801808169
:104C80008E7F8083888180618883DF91CF911F919F
:104C90000F910895E8EDF0E080818F7E8083E7ED4D
:104CA000F0E080818160808384E082BF81E0809336
:104CB000E8020C940726E8EDF0E080818E7F808387
:104CC0001092E20008951092DA001092E100089527
:104CD0001F920F920FB60F9211242F933F934F9371
:104CE0005F936F937F938F939F93AF93BF93EF9354
:104CF000FF938091E10082FF0BC08091E20082FF70
:104D000007C08091E1008B7F8093E1000E942B22FD
:104D10008091DA0080FF1FC08091D80080FF1BC007
:104D20008091DA008E7F8093DA008091D90080FF35
:104D30000DC080E189BD82E189BD09B400FEFDCFCF
:104D400081E08093E9020E94F22105C019BC109213
:104D5000E9020E9404228091E10080FF19C0809145
:104D6000E20080FF15C08091E2008E7F8093E20018
:104D70008091E20080618093E2008091D80080629F
:104D80008093D80019BC85E08093E9020E9411222B
:104D90008091E10084FF30C08091E20084FF2CC04C
:104DA00080E189BD82E189BD09B400FEFDCF80911B
:104DB000D8008F7D8093D8008091E1008F7E809312
:104DC000E1008091E2008F7E8093E2008091E2001A
:104DD00081608093E2008091E502882311F084E0F5
:104DE00007C08091E30087FD02C081E001C083E03D
:104DF0008093E9020E941D228091E10083FF29C077
:104E00008091E20083FF25C08091E100877F80933D
:104E1000E10082E08093E9021092E5028091E100D6
:104E20008E7F8093E1008091E2008E7F8093E2008C
:104E30008091E20080618093E20042E060E080E0E7
:104E40000E9466258091F00088608093F0000E94A7
:104E50000B22FF91EF91BF91AF919F918F917F9125
:104E60006F915F914F913F912F910F900FBE0F90D7
:104E70001F9018951F920F920FB60F9211242F9327
:104E80003F934F935F936F937F938F939F93AF93D2
:104E9000BF93CF93DF93EF93FF93C091E900CF705F
:104EA0008091EC00D82FD17080FDD0E81092E900FD
:104EB0008091F000877F8093F00078940E947E2795
:104EC0001092E9008091F00088608093F000CD2B73
:104ED000CF70C093E900FF91EF91DF91CF91BF9127
:104EE000AF919F918F917F916F915F914F913F9182
:104EF0002F910F900FBE0F901F9018951F93CF9377
:104F0000DF93CDB7DEB7AA970FB6F894DEBF0FBE1A
:104F1000CDBFEAEEF2E08091F100819322E0E23F22
:104F2000F207C9F70E9485228091E80083FF2EC115
:104F30008091EA029091EB02492F50E04A305105EE
:104F400008F024C1FA01EE59FF4F0C94192980385A
:104F500021F0823809F01AC108C08091E6029091D0
:104F6000E702992389F082600FC08091EE028F7072
:104F7000873008F00BC18093E9008091EB0085FB3E
:104F8000882780F91092E9009091E800977F90932C
:104F9000E8008093F1001092F100D1C0282F2D7FFE
:104FA00009F0F4C0882319F0823061F0EFC08091DD
:104FB000EC02813009F0EAC0933009F080E0809380
:104FC000E7022EC08091EC0281112AC08091EE028E
:104FD0008F702FEF280F263008F0D8C08093E9009B
:104FE0002091EB0020FF1CC0933021F48091EB0056
:104FF000806214C09091EB0090619093EB0021E0EF
:1050000030E0A90102C0440F551F8A95E2F7409392
:10501000EA001092EA008091EB0088608093EB0038
:105020001092E9008091E800877F8093E8000E9459
:105030009B25ACC08111AAC01091EC021F77809112
:10504000E3008078812B8093E3008091E800877FE4
:105050008093E8000E949B258091E80080FFFCCFB0
:105060008091E30080688093E300111102C082E028
:1050700001C083E08093E90289C08058823008F043
:1050800085C08091EC029091ED028C3D53E0950734
:1050900079F583E08A838AE289834FB7F894DE0149
:1050A000139620E03EE051E2E32FF0E050935700EA
:1050B000E49120FF03C0E295EF703F5FEF708E2F09
:1050C00090E0EA3010F0C79601C0C0968D939D9392
:1050D0002F5F243149F74FBF8091E800877F80938D
:1050E000E8006AE270E0CE0101960E94A72416C093
:1050F0006091EE027091EF02AE014F5F5F4F0E9430
:10510000EE23BC01892B09F441C09091E800977F00
:105110009093E80089819A810E9405258091E8009A
:105120008B778093E80032C0803881F58091E80069
:10513000877F8093E8008091E5028093F100809161
:10514000E8008E7772CF811121C08091EC0290919E
:10515000ED0299270297D4F48091E800877F80932D
:10516000E8008091EC028093E5020E949B258091EB
:10517000E502811106C08091E30087FD02C081E055
:1051800001C084E08093E9020E946C228091E800D3
:1051900083FF0AC08091E800877F8093E8008091B8
:1051A000EB0080628093EB00AA960FB6F894DEBF06
:1051B0000FBECDBFDF91CF911F910895CF93809106
:1051C000E9028823A1F0C091E900CF709091EC0032
:1051D000892F817090FD80E8C82B1092E9008091A2
:1051E000E80083FD0E947E27CF70C093E900CF9135
:1051F0000895991B79E004C0991F961708F0961B33
:10520000881F7A95C9F78095089597FB072E16F4A5
:10521000009407D077FD09D00E941F2907FC05D014
:105220003EF4909581959F4F0895709561957F4FBD
:105230000895EE0FFF1F0590F491E02D0994AA1B2D
:10524000BB1B51E107C0AA1FBB1FA617B70710F071
:10525000A61BB70B881F991F5A95A9F780959095A3
:10526000BC01CD010895FB01DC0104C08D910190CA
:10527000801921F441505040C8F7881B990B0895BC
:10528000F999FECF92BD81BDF89A992780B508950E
:10529000A8E1B0E042E050E00C947429262FF9997F
:1052A000FECF92BD81BDF89A019700B4021639F085
:1052B0001FBA20BD0FB6F894FA9AF99A0FBE089556
:1052C0000396272F0E944F290E944E29252F0E94C6
:1052D0004F29242F0C944F290196272F0E944F29E4
:1052E0000C944E29DC01CB01FC01F999FECF06C0DC
:1052F000F2BDE1BDF89A319600B40D924150504094
:08530000B8F70895F894FFCFFF
:10530800C8007C02280850011E0A1401702193214C
:105318007421EE21EA21732101E200E900EA00B5D7
:1053280000B600B700CD008301CC008A0192019439
:10533800012102230224022502260227022A02B39F
:1053480000B4006F007000818283E200E900EA0087
:10535800B500B600B700CD008301CC008A019201E8
:1053680094012102230224022502260227022A028E
:10537800B300B4006F00700081828330F4F73133DA
:105388003236F0F16795373534C666949091933F7D
:105398003F3F006D6B5F64656C6179006D6B5F69A1
:1053A8006E74657276616C006D6B5F6D61785F73AA
:1053B80070656564006D6B5F74696D655F746F5FC0
:1053C8006D6178006D6B5F776865656C5F6D61789E
:1053D8005F7370656564006D6B5F776865656C5FAA
:1053E80074696D655F746F5F6D617800407B22B092
:0C53F8000A350A130AB809D109EA0900B5
:00000001FF
